:020000040000FA
:0400000000007C2858
:040004000034003490
:080008008B13F000030E8301CD
:10001000F1000A08F2008A011A08BC008C123B1891
:100020006628BA1B3A283008840031088407000883
:100030003C02031D2528B10A05303102031D262884
:10004000B101B901FF30BA007528B1013808840048
:100050003908840700083C02031D3828B90A053016
:100060003902031D7528B101B901FF30BA007528A6
:10007000B90175283C08BA00FF30BB0000308A0087
:100080003A080F395120CD004D0803194F28BD0102
:10009000D201CD1F7528CD132808D2007528D81796
:1000A0007528D40000308A005408820700340434D4
:1000B0008434003400340034003400340034053417
:1000C000013400340034003400340034D208031901
:1000D0006B28D2037528400884003D0884073C083B
:1000E0008000BD0ACD0B7528D81772088A00710EE2
:1000F0008300F00E700E09004130C000BD01C10147
:10010000C201C301C401C501C601C701C801203035
:10011000B8008312B90138088400390884078316AF
:100120009B001C141A0883128000B90A0F30390290
:10013000031D8B284730B2005230B3005030B4005A
:100140003030B5003030B6003230B000B101293067
:10015000B800B901BA01BB01BD01D80107309F0049
:10016000831607308600831286011830D600861762
:1001700000008613D60BB7288616831640309900E8
:10018000043098008312903098008B170B17831659
:100190008C168312D81BCD28CA28BD01BB010030A4
:1001A0008A003A080F39D73E03188A0A82007C2851
:1001B000EA28EA28E728E728E728E728E728E728C1
:1001C00024291929E728E728E728E728E728BA019A
:1001D000D801CA2886120430D600410ED7000D215E
:1001E0000830D6004208D7000D210430D600430E57
:1001F000D7000D210830D6004408D7000D21411E3C
:100200000329861504298611431E08290616092983
:1002100006128616BA01D801CA288613D71F1229DA
:100220000617132906138617D70DD60B0D2986132B
:1002300008004108A8000830D1002830D000013063
:10024000BE00BA01D80136294108A9004208AA0017
:100250004308AB004408AC004508AD000930D100AC
:100260002930D0000530BE00BA01D8015008840002
:10027000000883169A008312510883169B009C1174
:100280001C1555309D00AA309D009C141C11831232
:100290008C1F48298C13D10AD00ABE0B3629B9010C
:0602A000BA01BB01CA28EF
:02400E00623F0F
:1042000000000000000000000000000000000000AE
:1042100000004400540053003000310020004400EE
:104220005400530043002000560031002E0030009F
:04423000300030002A
:00000001FF
